:020000040000FA
:020000002228B4
:08000800A0000308A1000B1188
:10001000AD0AAD1D1428AD012E17AE0A2E1D1428F1
:10002000F330AE052E16B92121088300A00E200E54
:020030000900C5
:040040000034003454
:0C004400831603308600FC3085008D30F0
:1000500081008312A0308B00051064000F309923BB
:10006000FF30A1236400C823031E41280230A800EA
:10007000AA01AB01AC01AD01AE01B001B801B901FB
:10008000BA010130AF006400A021A70000308A004F
:1000900027080F3982072A299628992851289C2851
:1000A000A2281430B9002F1D2A293008A400A40B5F
:1000B0006228AF1D5D28AF119C28AF120A23AF152F
:1000C000BA019C28A40B6A282F1E68282F129C288E
:1000D0002F169C28A40B6F28AF160A239C28A40B6C
:1000E00075282F142A3041229C286400A021A700E3
:1000F0002708031D8F282E1F75282E136400C82380
:10010000AE1C8D286400E830A123FC30A123BA3056
:10011000A123EE30A123E830A1232E12752803304D
:100120002706031D9C2800308A0022282F1D051455
:100130002A292F1D05102A2964002F142F1102309F
:10014000A8002A291430B9002F1DB0012F15B00ABC
:100150006400C8233008A400A40BCA28AF1DBE2821
:100160006400E830A123FC30A123BB30A123003080
:10017000A123BA30A123AF30A1232A2964005E3025
:10018000A123E930A1230030A123BA30A123AF304D
:10019000A1232A29A40BF4282F1EE0286400EE30A6
:1001A000A123E930A1230030A123AE30A123BA302E
:1001B000A123EE30A123A830A123BB30A1232A29FB
:1001C0006400D630A123BE30A123AF30A12300307C
:1001D000A123AE30A123BA30A123EE30A123A83051
:1001E000A123BB30A1232A29A40B082964005E3077
:1001F000A123E930A1230030A123AE30A123BA30DE
:10020000A123EE30A123A830A123BB30A1232A29AA
:10021000A40B182964005E30A123E930A12300302B
:10022000A1231E30A123BE30A123E930A1232A2916
:10023000A40B26296400E830A123FC30A123BA30A6
:10024000A123EE30A123E830A1232A296400013044
:10025000B000AE2864002E1F43282E132E1E8029C6
:100260002E12B90B37292F142F110230A800640069
:10027000AE1E8029AE1264002F1E8029AF1D5C299E
:100280003430B8000630A4002B08B5003A0EB60092
:10029000360DE039B6002C081F39B6043E30640034
:1002A000F3227F393502031D5B293F306400F322BE
:1002B00036020319AF1164290030B8001A30A400C7
:1002C0002B08B5002C08B60038086400F322A30000
:1002D000B700380A6400F322B70403197C293606F4
:1002E000031D7C2923087F393506031D7C29A31FA4
:1002F0007B2905147C2905100230B807A40B64295A
:100300002F1943280301640099232F1E97292A30AF
:100310006400E5210301AF1990296400A12392290B
:100320003A0AAE239A30051C1030A1234328AE1C94
:1003300087296400C82343280301A12B0130A12B86
:10034000A4017F30A300A40A8600A300231DAD29C9
:10035000861CB1290314230CA329A61BA601A617EA
:100360000034A61326082406031900342408A60026
:1003700008006400AA0A2A080F39093C0318E42976
:100380000630AA0760302A02031CE429AA01AE162F
:10039000AB0A2B080F39093C0318E4290630AB07D8
:1003A00060302B02031CE429AB01AC0A18302C0688
:1003B0001F39031DE429BA0A20302C07E039AC00AC
:1003C000E0302C060319AC010800023E8400280826
:1003D0002E180301A9001F300005EC3E031CF32971
:1003E000A4000230FC290A3E031CF929A4000130B4
:1003F000FC290A3EA4000301A91B9C21A91FAE23CE
:100400002408A91C082A291B9C21291FAE230C2A79
:10041000291B9E21291FB7238403000EA91A9C21A2
:10042000A91EAE230008A91C1A2A291A9C21291EDC
:10043000AE231E2A291A9E21291EB7238403A91937
:100440002E2A2F1C282A000EAE230008AE23332AA2
:1004500000089A3003191030A123332A03012F1802
:10046000A1230301A1230301A123840A840A000E0E
:10047000A400240C0739013E29199C21291DAE2313
:1004800008006400B10084000008B200840A00087B
:10049000B300840A0008B4008030A8006400A021E2
:1004A000A70002308A0027080F3982075C2A7C2ABD
:1004B000812AE02AF12A772A2E1F4E2A2E132E1E79
:1004C000712A2E122F1C712A6400B20A32080F39C9
:1004D000093C0318712A0630B20760303202031853
:1004E000B2010301992332306400E5214E2A031042
:1004F000A80D0318A80C712A0310A80CA818A80DA1
:10050000712AA81B8E2A281B9A2AA81AB92A281AE7
:10051000C32AA819CD2A2819D62A712A1F303405D2
:100520000A3EA300E23E0318A300E0303405230492
:10053000B400712A640034081F39EC3E031CA32A5E
:10054000A4001430AC2A0A3E031CA92AA4000A30D5
:10055000AC2A0A3EA4000301A300A40A2408F63E24
:100560000318A4012308A407E03034052404B400D0
:10057000712A1030B307330E0F39053C0318712A66
:100580000F30B305712A0130B30733080F39093C26
:100590000318712AF030B305712A2F1CD12AB20139
:1005A000712A0301321CFF30B200712A2030B407D7
:1005B000E0303406E039031D712A2030B407712A77
:1005C000640034081F39183CE030031CB4053108BE
:1005D000840032088000840A33088000840A3408CA
:1005E0008000A801080089008316081483120808F7
:1005F000080088002308890083168B1308155530DE
:100600008900AA30890088148B178818052B881058
:10061000831208000301AF1E3430B8006400C82301
:100620006F2B6400A021A700A70B242B02303807F2
:10063000B800AF1E1F2B333C031CB8016F2B3F3C8F
:100640003430031CB8006F2BA70B372B6400C82372
:10065000353041223808A300360835188038640048
:10066000F922380AA30037086400F9226F2BA70B80
:10067000562B6400030199230A30A1230301A1230F
:100680000A30A1230301A1230A30A1230301A123DE
:100690000A30A1230301A1233808A3000301640049
:1006A000F922A30A03016400F9226F2BA70B592B2F
:1006B0000800A70B6B2BAF1E632BFE30B807323040
:1006C000B81BB8006F2BFE30B807CC3038073E306F
:1006D000031CB8006F2B2E1F112B2E137B2B3808F9
:1006E0006400F322B600380A6400F322B700B501B3
:1006F000B61BB503B613030199230310380C64002D
:10070000D3232F100301A12335306400E521112BE1
:100710008200EE340634F234D6341E34DC34FC3439
:100720008634FE34DE34BE347C34E8347634F83437
:10073000B8340F39A300230E8600061185148510E6
:100740000800A300F0398600061585148510230ED5
:10075000F039860006158514851008000F39893E8A
:10076000A30003308A0023088823A12308000F393F
:10077000893EA30003308A00230888230138A1237F
:100780000800A400240E0F39AE2324080F39AE2B25
:100790000A30A400030199230301A123A40BCC2B4D
:1007A000030199230800A301A4000A302402031CBA
:1007B000DB2BA30AD42B2308AE2324080F39893E50
:0E07C000A30003308A00230888230138A12BF0
:02400E00F43F7D
:00000001FF
